:020000040800F2
:10000000002000209D210008650E0008670E0008F2
:1000100000000000000000000000000000000000E0
:10002000000000000000000000000000690E000851
:1000300000000000000000006B0E00086D0E0008BC
:10004000ED210008ED210008ED210008ED21000858
:10005000ED210008ED210008ED210008ED21000848
:10006000ED210008ED210008ED210008ED21000838
:10007000ED210008ED21000800000000ED2100083E
:1000800000000000ED21000800000000000000005A
:10009000ED21000800000000ED210008ED2100081E
:1000A000ED210008ED210008ED210008ED210008F8
:1000B000ED210008ED210008ED210008ED210008E8
:1000C00010B5064C2378002B07D1054B002B02D02E
:1000D000044800E000BF0123237010BD7000002021
:1000E000000000008C2B0008044B10B5002B03D03F
:1000F0000349044800E000BF10BDC04600000000F6
:10010000740000208C2B0008002243088B4274D31B
:1001100003098B425FD3030A8B4244D3030B8B4208
:1001200028D3030C8B420DD3FF22090212BA030C11
:100130008B4202D31212090265D0030B8B4219D3F2
:1001400000E0090AC30B8B4201D3CB03C01A524112
:10015000830B8B4201D38B03C01A5241430B8B425A
:1001600001D34B03C01A5241030B8B4201D30B0343
:10017000C01A5241C30A8B4201D3CB02C01A52416A
:10018000830A8B4201D38B02C01A5241430A8B422D
:1001900001D34B02C01A5241030A8B4201D30B0216
:1001A000C01A5241CDD2C3098B4201D3CB01C01A30
:1001B000524183098B4201D38B01C01A524143093A
:1001C0008B4201D34B01C01A524103098B4201D328
:1001D0000B01C01A5241C3088B4201D3CB00C01A95
:1001E000524183088B4201D38B00C01A524143080D
:1001F0008B4201D34B00C01A5241411A00D2014632
:10020000524110467047FFE701B5002000F0F0F8BA
:1002100002BDC0460029F7D076E7704703460B437E
:100220007FD4002243088B4274D303098B425FD3EF
:10023000030A8B4244D3030B8B4228D3030C8B421B
:100240000DD3FF22090212BA030C8B4202D3121201
:10025000090265D0030B8B4219D300E0090AC30BD6
:100260008B4201D3CB03C01A5241830B8B4201D383
:100270008B03C01A5241430B8B4201D34B03C01A6C
:100280005241030B8B4201D30B03C01A5241C30AE4
:100290008B4201D3CB02C01A5241830A8B4201D355
:1002A0008B02C01A5241430A8B4201D34B02C01A3F
:1002B0005241030A8B4201D30B02C01A5241CDD2E4
:1002C000C3098B4201D3CB01C01A524183098B422F
:1002D00001D38B01C01A524143098B4201D34B0118
:1002E000C01A524103098B4201D30B01C01A52417B
:1002F000C3088B4201D3CB00C01A524183088B4202
:1003000001D38B00C01A524143088B4201D34B00EA
:10031000C01A5241411A00D201465241104670475C
:100320005DE0CA0F00D04942031000D34042534061
:1003300000229C4603098B422DD3030A8B4212D321
:10034000FC22890112BA030A8B420CD38901921153
:100350008B4208D3890192118B4204D389013AD090
:10036000921100E08909C3098B4201D3CB01C01A65
:10037000524183098B4201D38B01C01A5241430978
:100380008B4201D34B01C01A524103098B4201D366
:100390000B01C01A5241C3088B4201D3CB00C01AD3
:1003A000524183088B4201D38B00C01A5241D9D2EB
:1003B00043088B4201D34B00C01A5241411A00D26C
:1003C0000146634652415B10104601D34042002B68
:1003D00000D54942704763465B1000D3404201B5E7
:1003E000002000F005F802BD0029F8D016E770479C
:1003F0007047C046002B11D1002A0FD1002900D12F
:10040000002802D00021C943081C07B4024802A1F9
:100410004018029003BDC046D9FFFFFF03B46846F1
:1004200001B5029800F030F8019B9E4602B00CBC6A
:100430007047C046F0B5CE46474615042D0C2E0039
:1004400080B50704140C3F0C9946030C7E435D43B2
:10045000674363437F19340CE4199C46A54203D9D2
:1004600080235B029846C4444B4643435143250CCA
:1004700036046544360C2404A4195B19591820006D
:100480000CBC90469946F0BDF0B54F464646D64660
:10049000C0B5040082B00D00914698468B422FD81B
:1004A0002CD04146484600F0B1F829000600200053
:1004B00000F0ACF8331A9C46203B9A4600D576E013
:1004C0004B46524693401F004B46624693401E00E7
:1004D000AF4228D825D05346A41BBD41002B00DADB
:1004E0007BE00022002300920193012352469340B7
:1004F0000193012362469340009318E08242D0D9D1
:1005000000220023009201930A9B002B01D01C6063
:100510005D600098019902B01CBC90469946A246C5
:10052000F0BDA342D7D90022002300920193634675
:10053000002BE9D0FB079846414672080A437B0826
:1005400066460EE0AB4201D1A2420CD8A41A9D41EE
:10055000012024196D410021013E24184D41002E37
:1005600006D0AB42EED9013E24196D41002EF8D1E0
:1005700000980199534600196941002B23DB2B0099
:100580005246D3402A006446E2401C005346150000
:10059000002B2DDB26005746BE4033002600674661
:1005A000BE403200801A994100900191ACE762464A
:1005B00020239B1A4A46DA406146130042468A408D
:1005C00017001F4380E7624620239B1A2A006646D5
:1005D0009A402300F3401343D4E7624620230021CE
:1005E0009B1A0022009101920122DA40019280E7D9
:1005F0002023624626009B1ADE402F00B046664646
:10060000B74046463B003343C8E7C04610B5002913
:1006100003D100F007F8203002E0081C00F002F8D7
:1006200010BDC0461C2101231B04984201D3000CBD
:1006300010391B0A984201D3000A08391B09984255
:1006400001D30009043902A2105C40187047C0466B
:10065000040302020101010100000000000000008B
:1006600002780B78002A03D0013001319A42F7D08A
:10067000D01A704770B5016002714371B02424062E
:10068000A4466144890A0D4EF46AFF250D400121FC
:10069000A9402143F16205682C6852000321914072
:1006A000C9430C402C600568EC682140E960006893
:1006B000C16893400B43C36070BDC0460010024048
:1006C00003681A69017901238B40134201D100208C
:1006D00070470120FCE70000F0B58BB01422002128
:1006E00005A801F0AFFD364BD96A04221143D96247
:1006F000D96A0A400192019AD96A80221143D962CB
:10070000D96A0A400292029ADA6A01242243DA6222
:10071000DA6A22400392039AD96A02221143D9620B
:10072000DB6A1A400492049BA026F6050022E02111
:10073000300000F07DFD234D00221021280000F044
:1007400077FD0022F721204800F072FD80239B01F5
:1007500005931E4B06930027079705A9280000F074
:10076000A1FC0F2305931A4B0693079705A92800B0
:1007700000F098FC2023059306940797089405A998
:10078000300000F08FFCC02305930694079708976C
:1007900005A9300000F086FC102305930694079706
:1007A000089705A9280000F07DFCF723059306941F
:1007B0000797089405A9044800F074FC0BB0F0BD3D
:1007C00000100240000800500004005000002110FA
:1007D0000000111010B50400C3061BD50122102122
:1007E000184800F025FDA3061AD50122202115483E
:1007F00000F01EFD630619D501224021114800F0CA
:1008000017FD64B2002C17DB002280210D4800F098
:100810000FFD10BD002210210A4800F009FDE2E79B
:1008200000222021074800F003FDE3E700224021D9
:10083000044800F0FDFCE4E701228021014800F0BB
:10084000F7FCE6E70004005070B50C00002826D144
:1008500000220121154800F0EBFC144D002202217A
:10086000280000F0E5FC2000FFF7B4FF012204217E
:10087000280000F0DDFC00220421280000F0D8FC54
:100880002401E0B2FFF7A6FF01220421280000F0B6
:10089000CFFC00220421280000F0CAFC70BD012218
:1008A0000121024800F0C4FCD7E7C0460004005014
:1008B00010B501000120FFF7C7FF10BD10B52021C2
:1008C0000020FFF7C1FF0A2000F08CFB2821002048
:1008D000FFF7BAFF012000F085FB08210020FFF799
:1008E000B3FF012000F07EFB01210020FFF7ACFFE9
:1008F000022000F077FB06210020FFF7A5FF012072
:1009000000F070FB0C210020FFF79EFF022000F09A
:1009100069FB10BD10B501210020FFF795FF0220F3
:1009200000F060FB10BD10B589014118C9B28039D3
:10093000C9B20020FFF788FF022000F053FB10BD72
:1009400010B5040002E00134FFF7B2FF2078002860
:10095000F9D110BD70B501608280C0231B069C4692
:100960006144890A0B4DEC6AFF231940FE3B1E00CF
:100970008E4031002143E962056829685200032452
:100980009440A14329600068016893400B430360D1
:1009900070BDC0460010024001684B69808801228A
:1009A000824013434B61704701684B698088012284
:1009B000824093434B61704770B505000C00254998
:1009C000FFF74EFE0300204328D0002B01D1012C5D
:1009D00028D021492800FFF743FE0300204325D0FB
:1009E000002B01D1012C25D01C492800FFF738FE2F
:1009F0000300204322D0002B01D1012C22D0184922
:100A00002800FFF72DFE030020431FD0002B08D144
:100A1000012C06D11348FFF7BFFF02E01248FFF791
:100A2000C3FF70BD1048FFF7B7FFFAE70F48FFF7A5
:100A3000BBFFF6E70D48FFF7AFFFF2E70C48FFF703
:100A4000B3FFEEE70A48FFF7A7FFEAE70548FFF71D
:100A5000ABFFE6E71C2C0008202C0008242C000823
:100A6000282C0008AC000020B4000020BC000020AE
:100A7000DC00002070B505000C00012A07D0E1B2AF
:100A80000020FFF750FF2800FFF75AFF70BDFFF767
:100A900041FFF4E730B585B001AC094B220023CB10
:100AA00023C2002001F04CFC01F0D4FB01F0F6FB66
:100AB0000321FFF799FC8900085905B030BDC046F5
:100AC000A42B000870B59CB0382200210EA801F0BC
:100AD000B9FB1422002109A801F0B4FB2422002153
:100AE000684601F0AFFB12490B68124A1A40802396
:100AF0001B0113430B6002250E950126119610234E
:100B00001293002418940EA800F0F0FB0F23099311
:100B10000A960B940C940D94002109A800F0AAFEEB
:100B200000950494684600F0B7FF1CB070BDC04645
:100B300000700040FFE7FFFFF0B5D6464F4680B596
:100B4000EBB000F029FAFFF7BDFFFFF7C5FD00F09D
:100B5000B1F9A14B1968012001431960D96803223A
:100B60009143D960DA680243DA609C4800F0EEF9FC
:100B7000A024E405052221009948FFF7EBFE062298
:100B800021009848FFF7E6FE072221009648FFF76C
:100B9000E1FE964C042221009548FFF7DBFE0D2272
:100BA00021009448FFF766FD002221009248FFF7DC
:100BB00061FD012221009148FFF75CFD904D02226A
:100BC00029009048FFF756FD8F4C03222900200092
:100BD000FFF750FD012200218C48FFF74BFFC82290
:100BE0005200002106A801F02DFBFFF767FE200050
:100BF000FFF766FDC0B200280CD000247D48FFF747
:100C00005FFDC0B200280BD000206BB00CBC914639
:100C10009A46F0BD01217E48FFF7CEFE0124EDE7A4
:100C2000012200217B48FFF725FF7B4F012138007F
:100C3000FFF7C2FEFA2000F0D5F9784E012130000E
:100C4000FFF7BAFEFA2000F0CDF9754D012128001A
:100C5000FFF7B2FEFA2000F0C5F900213800FFF7D7
:100C6000ABFEFA2000F0BEF900213000FFF7A4FE31
:100C7000FA2000F0B7F900212800FFF79DFEFA20C6
:100C800000F0B0F9002C15D0012200216548FFF7D3
:100C9000F1FE002201216448FFF7ECFE00250195DA
:100CA000012D0DD1002CAFD0012200215F48FFF7AC
:100CB000E1FEA9E7012200215D48FFF7DBFEEDE739
:100CC000FFF7E8FE01998B0006AA98504F1C2E00F2
:100CD00013E0B20006ABD358012100931800FFF7D0
:100CE0006BFEFA20400000F07DF900210098FFF72C
:100CF00063FE642000F076F90136BE42E9DB012292
:100D000000214C48FFF7B6FEA9463B48FFF7D8FC48
:100D1000C6B23A48FFF7D4FCC3B29A463948FFF747
:100D2000CFFCC0B2002E11D05346002B2DD000288E
:100D3000EBD13B4E01213000FFF73EFEC82000F012
:100D400051F900213000FFF737FE0BE0324E012150
:100D50003000FFF731FEC82000F044F900213000D8
:100D6000FFF72AFE32784B469B0006A95B581B789A
:100D70009A4217D12B0001229446E1444F4527DDCA
:100D80009342C2D11D0001978AE7244E0121300011
:100D9000FFF712FEC82000F025F900213000FFF710
:100DA0000BFEDFE7012200212348FFF763FE01224B
:100DB00000212248FFF75EFE019A214903A801F0B5
:100DC0009FFA0022012103A8FFF754FE0123D2E776
:100DD0001D00019764E7C046001002400024F400A3
:100DE000AC000020B4000020BC000020000800502F
:100DF000DC0000209C000020CC000020D40000205B
:100E0000001C0050A4000020C40000202C2C00086E
:100E1000282C0008382C00081C2C0008202C000866
:100E2000242C0008442C00084C2C00087C2C0008C2
:100E3000502C0008582C0008642C0008702C000866
:100E4000782C000870470000054B5A6B01210A43BB
:100E50005A63996B802252050A439A637047C046D1
:100E600000100240FEE7FEE77047704710B500F043
:100E7000A7F810BD10B503000B4A1268002A08D06D
:100E8000094A1068C3186A46934206D8064A136096
:100E900010BD054A05491160F2E701F0A9F90C23DC
:100EA000036001204042F3E78C0000207001002025
:100EB0007047000010B50C480C4B0360E1235B0247
:100EC000436000238360C36003610C22426183613D
:100ED000C3610362436201F02BF9002800D110BD09
:100EE000FFF7B0FFFBE7C046E400002000440040ED
:100EF00010B586B004001422002101A801F0A2F967
:100F00002268104B9A4201D006B010BD0E4B996B6F
:100F1000802292020A439A63D96A01221143D9625C
:100F2000DB6A1A400092009B0C2301930A3B029358
:100F30000133049301330593A02001A9C00500F0FB
:100F4000B1F8E1E7004400400010024010B5040091
:100F50000F4B1978FA208000FFF7D6F801000D4BEF
:100F60001868FFF7D1F800F081F800280DD1032CA4
:100F700001D901200AE0013000222100404200F0A6
:100F800043F8034B5C60002000E0012010BDC04628
:100F9000040000200000002010B5084A136840211A
:100FA0000B4313600020FFF7D1FF041E02D0012481
:100FB000200010BDFFF748FFFAE7C04600200240BE
:100FC000034A1168034B1B785B1813607047C046D7
:100FD0006801002004000020014B18687047C046DB
:100FE0006801002070B50400FFF7F6FF0500631CE0
:100FF00002D0044B1B78E418FFF7EEFF401BA04221
:10100000FAD370BD0400002070B5002811DB8308FE
:10101000144DC0339B005C5903221040C000FC32C9
:1010200016008640B44389010A40824022435A5147
:1010300070BDC0B20F230340083B9B0806339B00E2
:10104000094A944663445D6803242040C000FF229F
:1010500014008440A543890111408140294359600F
:10106000E6E7C04600E100E000ED00E001380A4B91
:1010700098420FD8094A50600948036A1B021B0AAC
:10108000C02109060B4303620023936007331360FA
:10109000002070470120FCE7FFFFFF0010E000E0A8
:1010A00000ED00E0F0B5CE46474680B5002333E0C2
:1010B000052600E00026AE4035003D430234A40082
:1010C000544EA551544C2568D4432E0026404F68F9
:1010D000FF0301D515432E004F4D2E606D682E0085
:1010E00026404F68BF0301D515432E004A4D6E6060
:1010F000AD682E0026404F68FF0201D515432E0033
:10110000454DAE60ED682C404E68B60201D52A43CD
:101110001400414AD46001330A681400DC4075D0E1
:1011200001249C402240F6D04D686E1E012E03D94A
:10113000112D01D0122D12D185685F000326BE400B
:10114000B5432E00CD68BD40354385604568A54355
:101150004C682609012434409C402C434460C768F5
:101160005E000324B440E443A44627408D68B540A4
:101170003D43C5604C68022C01D0122C10D1DC0814
:101180000834A400A146275807251D40AD000F24B0
:10119000AC40A7430C69AC4025003D434C4625506C
:1011A00005686446254003244F683C40B4402C4306
:1011B00004604C68E400AED5184D6C6B01263443D6
:1011C0006C639C08A51CAD00124EAF5903261E404F
:1011D000B5000F26AE40B743A026F605B04200D1B9
:1011E00068E70F4EB0420BD00E4EB0420AD00E4E02
:1011F000B04209D00D4EB04200D159E706265AE759
:10120000012658E7022656E7032654E70CBC904611
:101210009946F0BD0000014000040140001002406A
:101220000004005000080050000C0050001C00504A
:10123000002A01D1816270478161FCE710B5264B1D
:10124000DA680C231340082B42D00C2B11D0042B4E
:1012500009D0214B5A68520B0723134001338020D9
:101260000002984010BD1C4B1B68DB0632D51B48A2
:10127000F8E7910C0F230B401949C85C920D03232A
:101280001A40541C144BDB68DB030DD4124B1B6853
:10129000DB0613D5114A00230021FFF7CBF822000B
:1012A0000023FFF7A7F8DDE70E4A00230021FFF730
:1012B000C1F822000023FFF79DF8D3E70A4A002374
:1012C0000021FFF7B7F822000023FFF793F8C9E7E2
:1012D0000448C7E70448C5E70010024000093D0084
:1012E000B02B000800127A000024F400F0B583B09F
:1012F000041E00D19BE2C14BDA680C251540DA6868
:101300008026760216400368DB0736D5082D2CD0E0
:101310000C2D28D063688022520293424DD0A02227
:10132000D202934250D0B54B1A68B5490A401A60B0
:101330001A68802149020A400192019A1A68B1494B
:101340000A401A606368002B4AD0FFF745FE070089
:10135000AA4B1B689B0310D4FFF73EFEC01B6428FA
:10136000F6D9032064E2002ED4D0A44B1B689B0363
:1013700003D56368002B00D15CE223689B0765D529
:10138000E368042D3CD00C2D38D0002B00D1B0E008
:101390009A490A680920824313430B60FFF71CFE39
:1013A0000600964B1B685B0700D599E0FFF714FE1B
:1013B000801B0228F5D903203AE2904A1168802365
:1013C0005B020B431360BDE78C4B19688022D2028D
:1013D0000A431A601968802252020A431A60B1E770
:1013E000FFF7FAFD0700854B1B689B03C5D5FFF788
:1013F000F3FDC01B6428F6D9032019E2002EC4D1E6
:101400007E4A1268520702D5002B00D114E27B4EAF
:1014100072687D490A40216909020A437260326894
:1014200009218A4313433360FFF708FFF26812096A
:101430000F231340754AD35CD840754B1860754B29
:101440001868FFF783FD002800D0F1E12368DB0670
:101450002DD5002D60D1694B1B689B0503D5E36931
:10146000002B00D1EAE1654A53686B490B40616A81
:101470000B43536053681B021B0A216A09060B4386
:101480005360636A590B013180231B028B40D16882
:1014900009090F220A405D498A5CD3405C4A136007
:1014A0005C4B1868FFF752FD002800D0C0E12368AC
:1014B0001B077DD56369002B67D0504A136D01214E
:1014C0000B431365FFF788FD06004C4B1B6D9B0714
:1014D0006ED4FFF781FD801B0228F6D90320A7E117
:1014E00046494B68484A13402269120213434B6035
:1014F000ACE7424A136801218B431360FFF76CFD90
:1015000006003E4B1B685B07A0D5FFF765FD801BFF
:101510000228F6D903208BE1E369002B22D0374A59
:10152000116880235B000B431360FFF755FD060035
:10153000324B1B689B0506D4FFF74EFD801B02282B
:10154000F6D9032074E12D4A536833490B40616A90
:101550000B43536053681B021B0A216A09060B43A5
:101560005360A4E7254A13682C490B401360FFF72A
:1015700033FD0600214B1B689B0598D5FFF72CFD1A
:10158000801B0228F6D9032052E11C4A136D012169
:101590008B431365FFF720FD0600184B1B6D9B075F
:1015A00006D5FFF719FD801B0228F6D903203FE17D
:1015B00023685B0700D48EE0104B9B6BDB001BD4D1
:1015C0000E4A916B80235B050B4393630126144BFA
:1015D0001B68DB0528D5A36880225200934237D0D0
:1015E000002B4DD1054B1A6D0C490A401A651A6D36
:1015F0000C490A401A6531E00026E8E70010024075
:10160000FFFFFEFFFFFFFBFFFFE0FFFFBC2B00081B
:101610000000002008000020FF1FFFFFFFFEFFFF6B
:1016200000700040FFFBFFFF884A116880235B00C9
:101630000B431360FFF7D0FC0700844B1B68DB05EE
:10164000C9D4FFF7C9FCC01B6428F6D90320EFE01A
:101650007F4A116D80235B000B431365A368002B49
:1016600028D0FFF7B9FC0700794B1B6D9B0530D4E0
:10167000FFF7B2FCC01B774B9842F5D90320D7E0A7
:10168000A022D200934209D0714B1A6D72490A40D0
:101690001A651A6D71490A401A65DFE76C4B196DBE
:1016A000013AFF3A0A431A65196D802252000A4333
:1016B0001A65D3E7FFF790FC0700654B1B6D9B0590
:1016C00007D5FFF789FCC01B624B9842F5D9032070
:1016D000AEE0012E21D023689B063CD5A369002BE8
:1016E00021D05B4B99680120014399605A6B0243FA
:1016F0005A635B4A116A80239B010B431362FFF715
:101700006BFC0600524B9B689B0724D4FFF764FCDC
:10171000801B0228F6D903208AE04D4A936B514979
:101720000B409363D7E74A4A936801218B43936048
:101730004B4A136A4C490B401362FFF74DFC0600FD
:10174000434B9B689B0706D5FFF746FC801B02288E
:10175000F6D903206CE0A36A002B00D170E00C2DB9
:1017600049D0022B12D03A4A136840490B4013600B
:10177000FFF732FC0400364B1B689B0139D5FFF79D
:101780002BFC001B0228F6D9032051E0304A1368D5
:1017900036490B401360FFF71FFC05002C4B1B68FC
:1017A0009B0106D5FFF718FC401B0228F6D9032041
:1017B0003EE02749CB682E4A1340E26A206B024381
:1017C000606B02431343CB600A6880235B041343BE
:1017D0000B60FFF701FC04001D4B1B689B0106D446
:1017E000FFF7FAFB001B0228F6D9032020E00020B7
:1017F0001EE000201CE0012B24D0154BDA6880236A
:101800005B021340E16A8B4201D0012010E0F0231B
:101810009B031340216B8B4201D0012008E0C023C1
:101820001B041A40636B9A420ED0012000E0012095
:1018300003B0F0BD0120FBE70120F9E70120F7E745
:101840000020F5E70120F3E70020F1E700700040F9
:101850000010024088130000FFFEFFFFFFFBFFFFA8
:1018600000000140FFFFFFEFFFDFFFFFFFFFFFFE74
:10187000FFFF02FF70B505000C00002800D1D1E089
:101880006A4B1A68012313408B4219D32B689B07BC
:1018900006D5674AD368F0218B43A9680B43D36010
:1018A0002B68DB077BD56B68022B20D0032B40D045
:1018B000012B44D05E4A126892051DD4012099E0A4
:1018C0005A4A136801218B4323431360FFF784FBBB
:1018D0000600564B1A6801231340A342D6D0FFF7E7
:1018E0007BFB801B534B9842F3D9032082E0504A84
:1018F0001268920300D497E04D49CA6803208243DE
:101900001343CB60FFF768FB06006B68022B1CD00B
:10191000032B28D0012B34D0454BDB680C221A4214
:101920003DD0FFF759FB801B424B9842F4D903206E
:1019300060E03F4A12689201DED401205AE03C4A3E
:1019400012685207D8D4012054E0394BDA680C23CE
:101950001340082B23D0FFF73FFB801B354B9842E9
:10196000F3D9032046E0324BDA680C2313400C2BEA
:1019700015D0FFF731FB801B2E4B9842F3D9032083
:1019800038E02B4BDA680C231340042B07D0FFF709
:1019900023FB801B274B9842F3D903202AE0234BDB
:1019A0001A6801231340A34225D82B685B0706D58C
:1019B0001F4AD36820490B40E9680B43D3602B686A
:1019C0001B0707D51A49CB681C4A13402A69D20065
:1019D0001343CB60FFF732FC154BDA6812090F2373
:1019E0001340174AD35CD840164B1860164B186842
:1019F000FFF7ACFA70BD0D4A136801218B432343F6
:101A00001360FFF7E9FA0600084B1A680123134038
:101A1000A342CAD0FFF7E0FA801B064B9842F3D9E5
:101A20000320E7E70120E5E70120E3E7002002408B
:101A30000010024088130000FFF8FFFFFFC7FFFF00
:101A4000BC2B00080000002008000020014B186893
:101A50007047C0460000002010B5FFF7F7FF044BA9
:101A6000DA68120A07231340024AD35CD84010BD3B
:101A700000100240CC2B000810B5FFF7E7FF044B25
:101A8000DA68D20A07231340024AD35CD84010BD5B
:101A900000100240CC2B000870B5040082231B010B
:101AA00002681A425AD0704B9B6BDB0000D593E062
:101AB0006D4A916B80235B050B43936301256B4B50
:101AC0001B68DB0500D489E0674B1A68C0239B03C1
:101AD0001A4061680B40934200D194E0C0239B02FE
:101AE0000A001A409A4200D195E05F4B1B6DC0225C
:101AF000920213401FD01140994202D022689206F0
:101B000008D4C0229202A1680A409A4213D02368E6
:101B10001B0510D5544B186D554A02401E6D80218F
:101B2000090331431965196D524E314019651A6523
:101B3000C30500D576E06368C02292021900114007
:101B4000914200D17EE048490B6DC022920260684C
:101B5000024013430B65012D00D17DE02368DB07B4
:101B600006D5414AD36C03218B43E1680B43D36410
:101B700023689B0706D53C4AD36C0C218B43216913
:101B80000B43D36423685B0706D5374AD36C3A49C5
:101B90000B4061690B43D36423681B0706D5324AA7
:101BA000D36C36490B40A1690B43D36423685B06B1
:101BB00006D52D4AD36C32490B40216A0B43D364BE
:101BC00023681B064ED5284AD36C2E490B40E16989
:101BD0000B43D364002070BD002570E7234A1168D1
:101BE00080235B000B431360FFF7F6F906001F4BE1
:101BF0001B68DB0500D567E7FFF7EEF9801B64285B
:101C0000F5D90320E7E7C0239B03A0680340934274
:101C100000D063E769E7144B1B689B0300D464E7BB
:101C20000120D8E7FFF7D8F906000F4B1B6D9B0585
:101C300000D580E7FFF7D0F9801B134B9842F4D909
:101C40000320C8E708490A6810480240C020800302
:101C5000034013430B6076E70A008B6B0C490B4083
:101C600093637BE70020B6E700100240007000405D
:101C7000FFFFFCFFFFFFF7FFFFF3FFFFFFCFFFFFBB
:101C8000FFFFFFFBFFFFF3FF88130000FFFFCFFF05
:101C9000FFFFFFEFD0B504000168836802691343BA
:101CA00042691343C26913430A68964802401343CA
:101CB0000B602268536894490B40E1680B43536002
:101CC000A1692268914B9A4201D0236A1943936813
:101CD0008F4803400B43936022688E4B9A4216D084
:101CE0008D4B9A4227D0894B9A4239D0102387498D
:101CF0008A4257D080221202E169914200D18CE0E1
:101D0000082B00D9F7E09B00844AD3589F46844BA8
:101D1000D96C03230B40012B09D0002B05D0022BDB
:101D20003AD0032B05D01023E1E70123DFE704239A
:101D3000DDE70823DBE77A4BD96C0C230B40042B3F
:101D40000AD005D9082B29D00C2B07D10823CEE7C0
:101D5000002B03D10023CAE70423C8E71023C6E7FA
:101D60006F4BDB6CC02109010B408021C9008B4205
:101D70000ED009D9802109018B4211D0C02109015F
:101D80008B4207D10823B2E7002B03D10023AEE733
:101D90000423ACE71023AAE70223A8E70223A6E75F
:101DA0000223A4E7022B2DD007D9042B30D0082B17
:101DB00000D090E08020000207E0002B00D08AE0F5
:101DC000FFF74AFE002800D187E0626853009B18A5
:101DD000834200D983E01303834200D281E0070EDF
:101DE000060250080021801979410023FEF702FB0A
:101DF0004C4BC2184C4B9A4200D974E02368D8600F
:101E0000002053E0464B1B68DB0604D44748DCE760
:101E1000FFF714FAD6E74648D7E7082B65D89B00AA
:101E2000444AD3589F46FFF717FE00285FD0400072
:101E300063685B08C0186168FEF766F983B2000446
:101E4000000C010010393C4A914252D80F229343B2
:101E50001A0040080723184010432368D860002068
:101E600024E0FFF709FEE0E72D4B1B68DB0607D4F3
:101E70002E48DCE7FFF7E2F9D7E780200002D6E73B
:101E80002B48D4E7FFF7E8FD002836D063685B08ED
:101E900018186168FEF738F90004000C0200103AC7
:101EA000254B9A422BD82368D86000200023636614
:101EB000A366D0BDFFF7E0FDE6E7194B1B68DB0624
:101EC00007D41A48E2E7FFF7B9F9DDE780200002FE
:101ED000DCE71748DAE70120E8E70020E6E7012021
:101EE000E4E70120E2E70120E0E70120DEE700204F
:101EF000DCE70120DAE70120D8E70020D6E701205F
:101F0000D4E7C046F369FFEFFFCFFFFF0048004072
:101F1000FFF4FFFF0038014000440040D42B0008CC
:101F20000010024000FDFFFFFFFC0F000024F40042
:101F300000093D00F82B0008EFFF0000436ADB07B3
:101F400006D5026853682C490B40816A0B435360E5
:101F5000436A9B0706D50268536828490B40C16A4B
:101F60000B435360436A5B0706D5026853682449F4
:101F70000B40016B0B435360436A1B0706D5026895
:101F8000536820490B40416B0B435360436ADB06A7
:101F900006D5026893681C490B40816B0B43936024
:101FA000436A9B0606D50268936818490B40C16BCB
:101FB0000B439360436A5B060BD502685368144970
:101FC0000B40016C0B43536080235B03026C9A420D
:101FD0000AD0436A1B0606D5026853680D490B40B8
:101FE000816C0B4353607047026853680A490B4089
:101FF000416C0B435360ECE7FFFFFDFFFFFFFEFF6B
:10200000FFFFFBFFFF7FFFFFFFEFFFFFFFDFFFFF94
:10201000FFFFEFFFFFFFF7FFFFFF9FFFF0B5C64693
:1020200000B505000C0017009846069E2B68DB697A
:1020300023401B1B5A425341BB423BD1731CF5D07A
:10204000FEF7CAFF4346C01AB04220D8002E1ED069
:102050002B681A685207E9D5DA691205E6D580229D
:1020600012011A622A68136814490B4013602A6827
:102070009368A331FF318B4393602023AB67EB67F9
:102080008022AB5054330022EA54032013E02A6824
:1020900013680A490B4013602A689368A331FF3123
:1020A0008B4393602023AB67EB6754330022EA54E1
:1020B000032000E0002004BC9046F0BD5FFEFFFF5F
:1020C00030B583B0040080230022C250FEF784FFA5
:1020D000050023681B681B070DD423681B685B077A
:1020E00016D42023A367E367002323667422A35436
:1020F000002003B030BD80210C4B00930300002270
:1021000089032000FFF78AFF0028E6D00320F0E7CC
:102110008021064B00932B000022C9032000FFF70B
:102120007DFF0028DDD00320E3E7C046FFFFFF016D
:1021300010B5041E2ED0836F002B21D02423A3675B
:102140002268136801218B4313602000FFF7A2FD72
:10215000012814D0636A002B18D1226853680E49F5
:102160000B405360226893682A218B439360226856
:10217000136829390B4313602000FFF7A1FF10BD3E
:1021800074330022C254FEF7B3FED7E72000FFF7F6
:10219000D5FEE2E70120F2E7FFB7FFFF0D488546D5
:1021A0000D480E490E4A002302E0D458C4500433AF
:1021B000C4188C42F9D30B4A0B4C002301E0136086
:1021C0000432A242FBD3FEF773FE00F017F8FEF7CD
:1021D000B3FCFEE70020002000000020700000207B
:1021E000C42C00087000002070010020FEE70000F1
:1021F000014B18687047C0460C00002070B50026DF
:102200000C4D0D4C641BA410A64209D1002600F011
:10221000BDFC0A4D0A4C641BA410A64205D170BD3A
:10222000B300EB5898470136EEE7B300EB589847F8
:102230000136F2E7BC2C0008BC2C0008BC2C0008BE
:10224000C02C000803001218934200D17047197087
:102250000133F9E70D4B70B51C680500A36B002B2B
:102260000FD1182000F098F8094BA0630360094BC8
:1022700001224360084B83600B23838100230261AA
:1022800043610022A36B1D615A6170BD0C000020E8
:102290000E33CDAB34126DE6ECDE0500124B10B5FB
:1022A0001C68A36B002B0FD1182000F075F80F4BA2
:1022B000A06303600E4B012243600E4B83600B232F
:1022C0008381002302614361A46B0B4A2069616929
:1022D0000A4BFEF7AFF80122002380185941206114
:1022E00061614800400810BD0C0000200E33CDABEA
:1022F00034126DE6ECDE05002D7F954C2DF451581F
:102300000EB400B50B499CB01DAB0290069007912E
:1023100004910948094904CB0591006802A9019379
:1023200000F04EF90023029A13701CB008BC03B0F1
:102330001847C046FFFFFF7F0C0000200802FFFF88
:102340001FB50B4B040000226946186800F012F814
:10235000002804DA01225242D31700920193009818
:102360000199002C01D02060616004B010BDC0460E
:102370000C000020002370B5064C05000800110079
:10238000236000F0FBFB431C03D12368002B00D02B
:102390002B6070BD6C01002010B5034B0100186864
:1023A00000F04EF810BDC0460C00002070B50500CE
:1023B000002910D00C1F2368002B00DAE418280035
:1023C00000F0ABFB1D4A1368002B05D1636014605D
:1023D000280000F0A3FB70BDA34209D92168601852
:1023E0008342F3D118685B6841182160EEE713005F
:1023F0005A68002A01D0A242F9D919685818A04297
:102400000BD120680918581819608242E0D1106871
:102410005268411819605A60DAE7A04202D90C23C9
:102420002B60D5E721686018824203D1106852689A
:102430004118216062605C60CAE7C04694000020D9
:10244000032370B5CD1C9D43083506000C2D1ED20C
:102450000C25A9421DD8300000F05FFB254A146806
:102460002100002919D1244C2368002B03D130000E
:1024700000F01AFB20602900300000F015FB431C1F
:102480002BD10C233000336000F048FB03E0002D1B
:10249000DFDA0C233360002070BD0B685B1B19D49E
:1024A0000B2B03D90B60CC18256003E04B688C42E2
:1024B0000DD11360300000F031FB200007220B30FB
:1024C000231D9043C31AE7D05A42E250E4E7636009
:1024D0000C00EFE70C004968C3E70323C41C9C43CE
:1024E000A042E1D0211A300000F0DEFA431CDBD11B
:1024F000C7E7C0469400002098000020F0B58E6821
:1025000085B007000C00039201939E423CD89023B3
:102510008A89DB001A4234D00325096923685B1AD3
:102520000293636902985D43EB0F5D19019B6D1087
:1025300001331B18AB4200D91D00530532D52900C9
:102540003800FFF77DFF061E09D10C233B604023B6
:102550000120A28940421343A38105B0F0BD029A35
:10256000216900F0BEFAA389144A1A40802313435C
:10257000A381029B2661F61826606561019EED1A13
:10258000A560019B9E4200D9019E320003992068FC
:1025900000F0B0FAA36800209B1BA36023689E197B
:1025A0002660DAE72A00380000F0B9FA061EE0D10A
:1025B00021693800FFF7FAFEC7E7C0467FFBFFFF3F
:1025C000F0B5A1B003901D008B890F0016001B060B
:1025D00011D50B69002B0ED14021FFF731FF386078
:1025E0003861002805D10C23039A0138136021B00B
:1025F000F0BD40237B61002308AC63612033637628
:102600001033A376079535002B78002B01D0252BAE
:1026100046D1AB1B05930CD0320039000398FFF76D
:102620006DFF431C00D1AEE06269059B9446634494
:1026300063612B78002B00D1A5E0012200235242D8
:10264000626004A9543252186E1C2360E360A360D8
:102650001370A36531780522534800F037FA751CD2
:1026600000281FD12268D30604D5532304A95B1880
:1026700020211970130704D5532304A95B182B21BB
:10268000197033782A2B16D0350000210A20E36810
:102690002A786E1C303A092A4ED9002918D010E049
:1026A0000135B1E7404B2268C01A01238340134330
:1026B00023602E00CEE7079B191D1B680791002B96
:1026C00001DB0B9304E05B42E360022313432360CE
:1026D0002B782E2B0AD16B782A2B35D1079B02350C
:1026E0001A1D1B680792002B2BDB09932F4E2978AC
:1026F0000322300000F0EAF9002806D04023801BB6
:102700008340226801351343236029780622284834
:102710006E1C217600F0DAF900283CD0254B002B06
:1027200025D10722079B0733934308330793636937
:10273000049A9B18636166E7434301219B183500A7
:10274000A6E701235B42D0E700230A201A000135E7
:10275000636029786E1C3039092903D9002BC5D054
:102760000992C3E74243012352183500F1E707AB52
:1027700000933A00104B2100039800E000BF049042
:10278000049B0133D3D1BB890D985B0600D42EE79F
:10279000012040422BE707AB00933A00064B210093
:1027A000039800F079F8EAE7802C0008862C0008EE
:1027B0008A2C000800000000FD240008F7B5150071
:1027C00001938A680B6900900C00934200DA1300B1
:1027D00022002B6043321278002A01D001332B6093
:1027E00023689B0602D52B6802332B6006272368DB
:1027F0001F4027D0230043331B785A1E9341226881
:10280000920630D42200019943320098089EB047C6
:10281000431C25D0062320682A68E1680340002570
:10282000042B03D18D1AEB43DB171D40A3682269EB
:10283000934201DD9B1AED180027BD4220D10020F4
:1028400010E00137E3682A689B1ABB42D2DD220000
:102850000123193201990098089EB047431CF0D11A
:1028600001204042FEBD3020E118433108702100B4
:102870005A1C45310978A218433202331170C1E75E
:10288000220001231A3201990098089EB047431C88
:10289000E6D00137D1E70000F0B589B004920A0014
:1028A00043320593039002920A7E0C000E9B6E2A1F
:1028B00000D186E01FD8632A33D008D8002A00D17F
:1028C0008CE0582A4DD0250042352A7030E0642A29
:1028D00001D0692AF7D1196825680A1D280629D56B
:1028E00008681A60002803DA2D23029A4042137008
:1028F0006B4E0A274FE0732A74D008D86F2A1FD076
:10290000702AE0D1202209680A43226003E0752A78
:1029100016D0782AD7D12200782145321170614E25
:1029200022E025001A684235111D196013682B70CA
:10293000012365E008681A606906D3D500B2D1E7C3
:1029400019682568081D186008682E0605D5544EBC
:1029500008276F2A1BD00A2719E06D06F7D580B229
:10296000F5E745314E4E0A7018682268011D00686F
:102970001960150621D5D30702D520231A432260FA
:102980001027002803D1202322689A4322602300C5
:10299000002243331A706368A360002B58DB0422C3
:1029A000216891432160002854D1029D002B5AD008
:1029B0002500337842352B7055E05506DBD580B2C3
:1029C000D9E71A680D68101D4969186013682E064A
:1029D00001D5196002E06D06FBD519800023029D28
:1029E00023614FE01A68111D1960156800216268A3
:1029F000280000F06BF8002801D0401B606063687D
:102A000023610023029A13703CE023692A00049991
:102A10000398059DA847431C3ED023689B0715D407
:102A2000079BE068984239DA180037E0220001235A
:102A3000193204990398059EB047431C2CD00135E8
:102A4000E368079A9B1AAB42F0DCE9E70025F7E759
:102A50000028ADD0029D3900FDF7DCFB735C013D21
:102A60002B700028F7D1082F09D12368DB0706D582
:102A700063682269934202DC3023013D2B70029B84
:102A80005B1B2361059B07AA00932100049B03980D
:102A9000FFF794FE431CB8D10120404209B0F0BDBD
:102AA000912C0008A22C0008002370B5064C0500EC
:102AB00008002360FEF7DEF9431C03D12368002BD6
:102AC00000D02B6070BDC0466C010020C9B28218D6
:102AD000904201D10020704703788B42FBD0013037
:102AE000F6E7002310B59A4200D110BDCC5CC45467
:102AF0000133F8E710B5884202D98B18984203D306
:102B0000002307E08B5C8354013AFBD210BDCC5C00
:102B1000C45401339A42FAD1F8E770477047F8B5C8
:102B200007000D001600002905D11100FFF788FCF1
:102B300004002000F8BD002A03D1FFF737FC340061
:102B4000F7E700F012F82C00B042F2D23100380062
:102B5000FFF776FC041EECD029003200FFF7C1FF1E
:102B600029003800FFF722FCE3E70B1F1B68181F42
:102B7000002B01DA0B58C0187047000058220120C2
:102B8000014B40421A6070476C010020F8B5C04606
:102B9000F8BC08BC9E467047F8B5C046F8BC08BCF7
:042BA0009E46704796
:102BA4001C2C0008202C0008242C00080304060810
:102BB4000C1018203000000000000000000000008D
:102BC40001020304060708090000000001020304CF
:102BD400841E0008B41E0008BA1E0008F61E000871
:102BE400C61E0008F61E0008F61E0008F61E0008A1
:102BF400CC1E0008261E0008621E0008681E00087D
:102C0400EA1E0008741E0008EA1E0008EA1E0008F6
:102C1400EA1E00087A1E0008520000005600000058
:102C24004A0000005300000053494D4F4E5F535477
:102C34004D3332004C4554275320474F2021000088
:102C44004D4F444520324A004A3121004D4F4445FE
:102C540020314A004120564F5553202100000000E6
:102C640047414D45204F56455220210053434F5272
:102C740045203A00256400004A322100232D302BE0
:102C84002000686C4C006566674546470030313269
:102C940033343536373839414243444546003031C0
:102CA400323334353637383961626364656600001F
:082CB400D4D7FF7F01000000EE
:042CBC00E900000823
:042CC000C100000847
:102CC40000002000010000000400000010000020AB
:102CD40000000000000000000000000000000000F0
:102CE40000000000000000000000000000000000E0
:102CF40000000000000000000000000000000000D0
:102D040000000000000000000000000000000000BF
:102D140000000000000000000000000000000000AF
:102D2400000000000000000000000000000000009F
:040000050800219D31
:00000001FF
